:100000000C942A001895000018950000189500001F
:100010000C94E01B1895000018950000189500003E
:10002000189500001895000018950000189500001C
:10003000189500001895000018950000189500000C
:1000400018950000189500001895000018950000FC
:10005000189500008FE58DBFC0E4E0E14E2E84E0EE
:100060008EBFD4E0F4E05F2EEEEFF3E0A0E6B0E068
:1000700088278D933197E9F70E941B19662478949D
:10008000E3E0F0E0A1E7B0E00E94F91CE4E0F0E07A
:10009000A4E7B0E00E94F91C8FEF8ABBD0988FEFE5
:1000A00087BB8FEF84BB80E081BB88E082BD85E0A9
:1000B00085BD89B7806489BF83E086B980EC87B944
:1000C0008CE00E9475190E94001981E783BF839B11
:1000D0000C9477008FEF8CBF87E080936E0088E0F0
:1000E00080936F008CE0809370000C949A00E0E0A5
:1000F000F0E0AEE6B0E00E94F91CE1E0F0E0AFE62F
:10010000B0E00E94F91CE2E0F0E0A0E7B0E00E945D
:10011000F91C02E010E0AFE6B0E04D9155270E94D7
:10012000D118A3EBB3E00D931C930091B30341E00E
:10013000041B0CBF0E9437180E94DA178FE711E0EA
:100140000E940F19EAE2FAE30E94F9188FEB11E01E
:100150000E940F19ECE3FAE30E94F918E1E0F0E0E5
:100160000E94121981E08093B1030091B103013123
:1001700018F011F00C94DA00E1EBF3E0A190BB244D
:10018000E3E0F0E0AA0CBB1CEA0DFB1DA1EBB3E021
:10019000AD90BB24A3E7B0E0AA0CBB1CAA0DBB1D0D
:1001A0000E94FB1CA1EBB3E08C918F5F8C9310F449
:1001B0000C94B50081E08093B1030091B103033644
:1001C00018F011F00C940701E1EBF3E0A190BB24CF
:1001D000E3E2F0E0AA0CBB1CAA0CBB1CEA0DFB1D61
:1001E000A1EBB3E0AD90BB24A4EBB1E0AA0CBB1C27
:1001F000AA0CBB1CAA0DBB1D94E00E94FC1CA1EB29
:10020000B3E08C918F5F8C9310F40C94DD00A4E428
:10021000B3E0EEE4FAE30E94761BA5E5B3E0E0E686
:10022000FAE30E94761BA6E6B3E0E2E7FAE30E9457
:10023000761BA7E7B3E0E4E8FAE30E94761B84E9C3
:10024000A7E7B3E08F930E94EA188F918D938827D8
:100250008C93A7E7B3E00E94EA18E0E9FAE30E9472
:10026000761BA8E8B3E0E6E9FAE30E94761B84E98E
:10027000A8E8B3E08F930E94EA188F918D938827A6
:100280008C93A8E8B3E00E94EA18E2EAFAE30E943D
:10029000761BA9E9B3E0E8EAFAE30E94761B84E959
:1002A000A9E9B3E08F930E94EA188F918D93882774
:1002B0008C93A9E9B3E00E94EA18E0E9FAE30E940E
:1002C000761BA7E9B0E0E4EBFAE30E94761BA8EA0C
:1002D000B0E0E6ECFAE30E94761BA9EBB0E0E8EDB3
:1002E000FAE30E94761BAAECB0E0EAEEFAE30E9481
:1002F000761BABEDB0E0ECEFFAE30E94761BACEEC0
:10030000B0E0EEE0FBE30E94761BADEFB0E0E0E290
:10031000FBE30E94761BAEE0B1E0E2E3FBE30E9468
:10032000761BAFE1B1E0E4E4FBE30E94761BA0E3BF
:10033000B1E0E6E5FBE30E94761BA1E4B1E0E8E66C
:10034000FBE30E94761BA2E5B1E0EAE7FBE30E9433
:10035000761BA3E6B1E0ECE8FBE30E94761BA4E782
:10036000B1E0EEE9FBE30E94761BA5E8B1E0E0EB2B
:10037000FBE30E94761BA6E9B1E0E2ECFBE30E94FE
:10038000761BA7EAB1E0E4EDFBE30E94761BC19A7D
:100390000E94DA17379A80EC806C87B90E947C1B28
:1003A000082F192F043F51E0150781E008F480E081
:1003B0008F9380EC806C87B90E947C1B082F192FCB
:1003C0000F3153E0150781E010F009F080E09F91B4
:1003D0008923882311F40C9401028FE711E00E9415
:1003E0000F19E6EEFBE30E94F9188FEB11E00E9473
:1003F0000F19E8EFFBE30E94F9180C94C7010C9465
:10040000550280EC806C87B90E947C1B082F192F45
:10041000003253E0150781E008F480E08F9380EC10
:10042000806C87B90E947C1B082F192F043853E079
:10043000150781E010F009F080E09F91892388235F
:1004400011F40C9435028FE711E00E940F19EAE0D5
:10045000FCE30E94F9188FEB11E00E940F19E8EFFE
:10046000FBE30E94F9180C94550280EC806C87B96C
:100470000E947C1B082F192F043853E0150718F031
:1004800011F00C9445020C9455028FE711E00E9484
:100490000F19ECE1FCE30E94F9188FEB11E00E94C8
:1004A0000F19EEE2FCE30E94F9183798C198E2E0D8
:1004B000F0E00E94121980E08093B20380E0809304
:1004C000BB03A0E6B0E00E94AE1BC498C7980E9490
:1004D000DA178FE711E00E940F19E0E4FCE30E94B5
:1004E000F9188FEB11E00E940F19E2E5FCE30E947E
:1004F000F91884E80E946F19EEE5FCE30E94F918F0
:100500000E94CB178C98AAEAB3E09C9194FF04C098
:10051000849910C09F7E9C93849B0CC084E69F931B
:1005200099270E94F9199F91849B04C090619C9324
:100530000E94BC0A8D98AAEAB3E09C9193FF04C084
:10054000859910C0977F9C93859B0CC084E69F93F0
:1005500099270E94F9199F91859B04C098609C93EC
:100560000E94DB0A0091B203013081E009F080E0D3
:100570008F93A0E3B0E00C9103FB81E00EF080E0EC
:100580009F918923882311F40C94C8020C9460076E
:100590000091B203023081E009F080E08F93A0E384
:1005A000B0E00C9103FB81E00EF080E09F91892385
:1005B000882311F40C94DE020C9442080091B203DB
:1005C000033081E009F080E08F93A0E3B0E00C916C
:1005D00003FB81E00EF080E09F918923882311F4D2
:1005E0000C94F4020C9436090091B203043081E0BB
:1005F00009F080E08F93A0E3B0E00C9103FB81E071
:100600000EF080E09F918923882311F40C940A0353
:100610000C9459030091B203053081E009F080E0A9
:100620008F93A0E3B0E00C9103FB81E00EF080E03B
:100630009F918923882311F40C9420030C94C408FF
:100640000091B203063081E009F080E08F93A0E3CF
:10065000B0E00C9103FB81E00EF080E09F918923D4
:10066000882311F40C9436030C94D00584E690E0B2
:100670000E94F9190C9482020E940C188FE711E075
:100680000E940F19E4E6FCE30E94F9188FEB11E0D9
:100690000E940F19E6E7FCE30E94F918F89480E045
:1006A00083BFC39A85B78F7D806685BF8895F89490
:1006B000FFCF8091AA0380688093AA0381E0809392
:1006C000BB030E94BF15ABEBB3E0AD90BB24A3E727
:1006D000B0E0AA0CBB1CAA0DBB1D0D911C910030F3
:1006E00050E0150711F00C9477030C94B1050E94AB
:1006F0000C188091AA038F7B8093AA03ADE7B0E02A
:100700000D911C91A3E8B0E04D915C91040F151F71
:10071000AEEAB3E00D931C93AEEAB3E00D911C91E9
:10072000A9E8B0E04D915C91040F151FAEEAB3E06B
:100730000D931C93AEEAB3E00D911C91AFE8B0E0CD
:100740004D915C91040F151FAEEAB3E00D931C931D
:10075000AEEAB3E00D911C91A5E9B0E04D915C913A
:10076000040F151FAEEAB3E00D931C93A5E7B0E0AC
:100770008D919C91A0E6B0E08D939C93A0E6B0E0B3
:100780000D911C91003050E0150718F011F00C94F9
:10079000CB030C9401048B98AAEAB3E09C9192FFDE
:1007A00004C0839910C09B7F9C93839B0CC084E6FC
:1007B0009F9399270E94F9199F91839B04C094608D
:1007C0009C930C945B0284E690E00E94F9198FE7F9
:1007D00011E00E940F19A7E9B0E00E94F3188FEB17
:1007E00013E00E940F19A8EFB3E0E0E6F0E00E94EA
:1007F000891C0E94F118E8E8FCE30E94F9180C94A7
:10080000BE03ADE7B0E00D911C91003050E015073C
:1008100018F011F00C940E040C945504ADE7B0E000
:100820008D919C91ACEAB3E08D939C930E943A1613
:100830000E94B5150091BB03033011F00C94220403
:100840000E94F8170E949116AAEAB3E08C9187FBE8
:1008500016F40C942D040C945B020091BB0304303D
:1008600011F00C941804ACEAB3E00D911C9141E036
:1008700050E0041B150BACEAB3E00D931C93AEEAF9
:10088000B3E00D911C9141E050E0041B150BAEEA62
:10089000B3E00D931C93ACEAB3E00D911C910030D2
:1008A00050E0150711F00C941604A3E8B0E00D9188
:1008B0001C91003050E0150718F011F00C94620400
:1008C0000C94AC04A3E8B0E08D919C91ACEAB3E049
:1008D0008D939C930E943A1685E08093BB030E94FF
:1008E000B5150091BB03063011F00C9479040E94F9
:1008F000F8170E949116AAEAB3E08C9187FB16F4D0
:100900000C9484040C945B020091BB03073011F03B
:100910000C946F04ACEAB3E00D911C9141E050E0FF
:10092000041B150BACEAB3E00D931C93AEEAB3E0E5
:100930000D911C9141E050E0041B150BAEEAB3E0B1
:100940000D931C93ACEAB3E00D911C91003050E084
:10095000150711F00C946A04A9E8B0E00D911C9100
:10096000003050E0150718F011F00C94B9040C9405
:100970000305A9E8B0E08D919C91ACEAB3E08D93BA
:100980009C930E943A1688E08093BB030E94B515A1
:100990000091BB03093011F00C94D0040E94F817A9
:1009A0000E949116AAEAB3E08C9187FB16F40C948E
:1009B000DB040C945B020091BB030A3011F00C9431
:1009C000C604ACEAB3E00D911C9141E050E0041B79
:1009D000150BACEAB3E00D931C93AEEAB3E00D91B6
:1009E0001C9141E050E0041B150BAEEAB3E00D93FF
:1009F0001C93ACEAB3E00D911C91003050E0150758
:100A000011F00C94C104AFE8B0E00D911C910030DE
:100A100050E0150718F011F00C9410050C945A05CD
:100A2000AFE8B0E08D919C91ACEAB3E08D939C93DC
:100A30000E943A168BE08093BB030E94B51500918B
:100A4000BB030C3011F00C9427050E94F8170E948C
:100A50009116AAEAB3E08C9187FB16F40C94320548
:100A60000C945B020091BB030D3011F00C941D053A
:100A7000ACEAB3E00D911C9141E050E0041B150B72
:100A8000ACEAB3E00D931C93AEEAB3E00D911C9178
:100A900041E050E0041B150BAEEAB3E00D931C934C
:100AA000ACEAB3E00D911C91003050E0150711F055
:100AB0000C941805A5E9B0E00D911C91003050E0B0
:100AC000150718F011F00C9467050C94B105A5E911
:100AD000B0E08D919C91ACEAB3E08D939C930E9421
:100AE0003A168EE08093BB030E94B5150091BB03BC
:100AF0000F3011F00C947E050E94F8170E94911699
:100B0000AAEAB3E08C9187FB16F40C9489050C9447
:100B10005B020091BB03003111F00C947405ACEA48
:100B2000B3E00D911C9141E050E0041B150BACEAC1
:100B3000B3E00D931C93AEEAB3E00D911C9141E03C
:100B400050E0041B150BAEEAB3E00D931C93ACEA26
:100B5000B3E00D911C91003050E0150711F00C949A
:100B60006F050E94DA178FE711E00E940F19E4E881
:100B7000FAE30E94F91884E90E946F19E0E9FAE3A8
:100B80000E94F9188FEB11E00E940F19E4E9FCE3D1
:100B90000E94F918E4E0F0E00E9412190C94C701D9
:100BA0000E940C188091AA038F7B8093AA0381E096
:100BB0008093BB0381E08093BF0381E08093C003F7
:100BC00080E08093C1034FEF5FEF6FEF7FEFABEB00
:100BD000B3E0AD90BB24A4EBB1E0AA0CBB1CAA0C03
:100BE000BB1CAA0DBB1D0D911D912D913C910E9426
:100BF000761C80E014F009F081E08F930091BB0334
:100C0000043681E008F080E09F918923882311F465
:100C10000C9482068FEB11E00E940F19E6EAFCE3C8
:100C20000E94F918EBEBF3E0A190BB24E4EBF1E0B8
:100C3000AA0CBB1CAA0CBB1CEA0DFB1DA8EFB3E061
:100C40000E94411B0E94F1188FE711E00E940F19CA
:100C5000EEEAFCE30E94F9180E94081AABECB3E03C
:100C60000E94F3188B98AAEAB3E09C9192FF04C00B
:100C7000839910C09B7F9C93839B0CC084E69F93B9
:100C800099270E94F9199F91839B04C094609C93BB
:100C90000C945B0284E690E00E94F919ECEBF3E01F
:100CA0000E94081BA0E1B0E04D915D916D917C9197
:100CB000ABEBB3E0AD90BB24A4EBB1E0AA0CBB1C42
:100CC000AA0CBB1CAA0DBB1D0D911D912D913C9131
:100CD0000E94761C11F00C942406009171000130E2
:100CE00011F00C9479060E94FF1784EF91E00E94A6
:100CF000F9190E94FF17ABEBB3E08C918F5F8C93D7
:100D00000C94E3050E94DA178FE711E00E940F1997
:100D1000E8EAFAE30E94F91884E90E946F19E0E911
:100D2000FAE30E94F9188FEB11E00E940F19E4E931
:100D3000FCE30E94F918E4E0F0E00E9412190C9420
:100D4000C7010E94DA178FEB11E00E940F19E6EB42
:100D5000FCE30E94F91881E08093B1030091B10394
:100D6000013118F011F00C94D406E1EBF3E0A190FE
:100D7000BB24E3E0F0E0AA0CBB1CEA0DFB1DA1EBD9
:100D8000B3E0AD90BB24A3E7B0E0AA0CBB1CAA0D56
:100D9000BB1D7BE70E94EA1CA1EBB3E08C918F5F47
:100DA0008C9310F40C94AE0681E08093B103009113
:100DB000B103033618F011F00C940207E1EBF3E0F5
:100DC000A190BB24E3E2F0E0AA0CBB1CAA0CBB1C64
:100DD000EA0DFB1DA1EBB3E0AD90BB24A4EBB1E0A9
:100DE000AA0CBB1CAA0CBB1CAA0DBB1D94E07BE784
:100DF0000E94EB1CA1EBB3E08C918F5F8C9310F4FD
:100E00000C94D706E0E0F0E0AEE6B0E07BE70E94AD
:100E1000E81CE1E0F0E0AFE6B0E07BE70E94E81C10
:100E2000E2E0F0E0A0E7B0E07BE70E94E81CE3E04E
:100E3000F0E0A1E7B0E07BE70E94E81CE4E0F0E02E
:100E4000A4E7B0E07BE70E94E81C0C945B020E94E0
:100E5000DA178FEB11E00E940F19E8ECFCE30E9417
:100E6000F91884E90E946F19E4EDFCE30E94F91877
:100E700081E08093B1030091B103033618F011F0C3
:100E80000C945A07A1EBB3E0AD90BB24A4EBB1E006
:100E9000AA0CBB1CAA0CBB1CAA0DBB1DE6E0FAE306
:100EA0000E949E1BA1EBB3E08C918F5F8C9310F49A
:100EB0000C943B07E2E0F0E00E9412190C945B02F4
:100EC0000E94170B0E94CB178C98AAEAB3E09C9162
:100ED00094FF04C0849910C09F7E9C93849B0CC097
:100EE00084E69F9399270E94F9199F91849B04C0DF
:100EF00090619C930E94170B8D98AAEAB3E09C9195
:100F000093FF04C0859910C0977F9C93859B0CC06C
:100F100084E69F9399270E94F9199F91859B04C0AD
:100F200098609C930E94360B8998AAEAB3E09C9142
:100F300091FF04C0819910C09D7F9C93819B0CC040
:100F400084E69F9399270E94F9199F91819B04C081
:100F500092609C930E9427118A98AAEAB3E09C9120
:100F600090FF04C0829910C09E7F9C93829B0CC00E
:100F700084E69F9399270E94F9199F91829B04C050
:100F800091609C930E948C0E0091BB03073011F07E
:100F90000C94E4078B98AAEAB3E09C9192FF04C0FA
:100FA000839910C09B7F9C93839B0CC084E69F9386
:100FB00099270E94F9199F91839B04C094609C9388
:100FC0000C9427070C943C080091BB03083011F0E7
:100FD0000C9404088B98AAEAB3E09C9192FF04C099
:100FE000839910C09B7F9C93839B0CC084E69F9346
:100FF00099270E94F9199F91839B04C094609C9348
:101000000C94A1060C943C080091BB03093011F02C
:101010000C9424088B98AAEAB3E09C9192FF04C038
:10102000839910C09B7F9C93839B0CC084E69F9305
:1010300099270E94F9199F91839B04C094609C9307
:101040000C943C030C943C088B98AAEAB3E09C9166
:1010500092FF04C0839910C09B7F9C93839B0CC01C
:1010600084E69F9399270E94F9199F91839B04C05E
:1010700094609C930C945B0284E690E00E94F919C2
:101080000C9464070E94860C0E94CB178C98AAEAE5
:10109000B3E09C9194FF04C0849910C09F7E9C9300
:1010A000849B0CC084E69F9399270E94F9199F9115
:1010B000849B04C090619C930E94860C8D98AAEA40
:1010C000B3E09C9193FF04C0859910C0977F9C93D7
:1010D000859B0CC084E69F9399270E94F9199F91E4
:1010E000859B04C098609C930E94A50C8998AAEAED
:1010F000B3E09C9191FF04C0819910C09D7F9C93A7
:10110000819B0CC084E69F9399270E94F9199F91B7
:10111000819B04C092609C930E9427118A98AAEA3E
:10112000B3E09C9190FF04C0829910C09E7F9C9375
:10113000829B0CC084E69F9399270E94F9199F9186
:10114000829B04C091609C930E948C0E8B98AAEAAB
:10115000B3E09C9192FF04C0839910C09B7F9C9345
:10116000839B0CC084E69F9399270E94F9199F9155
:10117000839B04C094609C930C945B0284E690E093
:101180000E94F9190C9446080E94370D0E94CB1753
:101190008C98AAEAB3E09C9194FF04C0849910C093
:1011A0009F7E9C93849B0CC084E69F9399270E940A
:1011B000F9199F91849B04C090619C930E94370D04
:1011C0008D98AAEAB3E09C9193FF04C0859910C062
:1011D000977F9C93859B0CC084E69F9399270E94E0
:1011E000F9199F91859B04C098609C930E94560DAD
:1011F0000091BB03033011F00C9418098B98AAEAF4
:10120000B3E09C9192FF04C0839910C09B7F9C9394
:10121000839B0CC084E69F9399270E94F9199F91A4
:10122000839B04C094609C930C945B020C943009E3
:101230008B98AAEAB3E09C9192FF04C0839910C0F6
:101240009B7F9C93839B0CC084E69F9399270E946D
:10125000F9199F91839B04C094609C930E94B809E4
:1012600084E690E00E94F9190C94C8080E94AA0D27
:101270000E94CB178C98AAEAB3E09C9194FF04C01B
:10128000849910C09F7E9C93849B0CC084E69F939E
:1012900099270E94F9199F91849B04C090619C93A7
:1012A0000E94AA0D8D98AAEAB3E09C9193FF04C016
:1012B000859910C0977F9C93859B0CC084E69F9373
:1012C00099270E94F9199F91859B04C098609C936F
:1012D0000E94C90D8998AAEAB3E09C9191FF04C0CD
:1012E000819910C09D7F9C93819B0CC084E69F9345
:1012F00099270E94F9199F91819B04C092609C9349
:101300000E9427118A98AAEAB3E09C9190FF04C03A
:10131000829910C09E7F9C93829B0CC084E69F9311
:1013200099270E94F9199F91829B04C091609C9318
:101330000E948C0E8B98AAEAB3E09C9192FF04C0A5
:10134000839910C09B7F9C93839B0CC084E69F93E2
:1013500099270E94F9199F91839B04C094609C93E4
:101360000C945B0284E690E00E94F9190C943A090F
:101370000E94DA178FE711E00E940F19EAEDFCE3F3
:101380000E94F9188FEB11E00E940F19ECEEFCE3BC
:101390000E94F9180E94CB170E94BE17C49A0091B0
:1013A0007100013011F00C94E5090E94DA178FE703
:1013B00011E00E940F19E6ECFAE30E94F9180E946E
:1013C000CB170E94BE170E94FF170091BB0301308C
:1013D00011F00C94470A0E94DA178FE711E00E947F
:1013E0000F19EEEFFCE30E94F91884E90E946F19CF
:1013F000E4E0FDE30E94F9180E94CB170E94BE179B
:101400000E940C180E94DA178FE711E00E940F1952
:10141000E0E1FDE30E94F9188FEB11E00E940F1943
:10142000EAE1FDE30E94F9188091AA038F7B809383
:10143000AA03A0E6B0E00E94AE1B0E94F817A0E34A
:10144000B0E00C9103FB0EF416C08FE71BE00E9486
:101450000F19A8EFB3E0E0E6F0E00E94891C0E94BB
:10146000F118ECE2FDE30E94F91884E690E00E9496
:10147000F9190C941F0A0E94DA178FE711E00E94F5
:101480000F19EEE2FDE30E94F9180C94AD0A0091E9
:10149000BB03023011F00C94AD0A0E94DA178FE7FB
:1014A00011E00E940F19E6E9FAE30E94F91884E9B5
:1014B0000E946F19E2EAFAE30E94F9188FEB11E03B
:1014C0000E940F19E0E4FDE30E94F9180E94CB1777
:1014D0000E94BE170E9400190E94DA178FE711E0E0
:1014E0000E940F19E2E5FDE30E94F91884E80E94CA
:1014F0006F19EEE5FDE30E94F918A0E6B0E00E9446
:10150000AE1B0E94F817A0E3B0E00C9103FB0EF0B5
:101510001CC00E94DA178FEB11E00E940F19E4E65D
:10152000FDE30E94F918A8EFB3E0E0E6F0E00E94C6
:10153000891C0E94F118ECE2FDE30E94F91884E690
:1015400090E00E94F9190C94830A8FE711E00E9441
:101550000F19E0E7FDE30E94F918C498C7980E94AC
:10156000DA178FEB11E00E940F19E2E8FDE30E9409
:10157000F9180E94CB170895A2EBB3E08C918F5F0E
:101580008C930091B203063080E010F009F081E006
:101590008F930091B203013081E008F080E09F91C9
:1015A000892B882311F40C94D80A81E08093B2032C
:1015B0000E94FA0A0895A2EBB3E08C9181508C93BB
:1015C0000091B203013081E008F080E08F93009138
:1015D000B203063080E010F009F081E09F91892B82
:1015E000882311F40C94F70A86E08093B2030E94DA
:1015F000FA0A08950E94DA178FE711E00E940F1986
:10160000A2EBB3E00D91112741E150E00E94491B8C
:10161000A3E3B3E0A00FB11F0E94F3188FEB11E01A
:101620000E940F19E2E8FDE30E94F9180895ABEB60
:10163000B3E08C918F5F8C930091BB03093080E005
:1016400010F009F081E08F930091BB03013081E03D
:1016500008F080E09F91892B882311F40C94330BC0
:1016600081E08093BB030E94550B0895ABEBB3E080
:101670008C9181508C930091BB03013081E008F084
:1016800080E08F930091BB03093080E010F009F0F7
:1016900081E09F91892B882311F40C94520B89E0EF
:1016A0008093BB030E94550B08950E94001900917E
:1016B000BB03013011F00C94750B0E94DA178FE711
:1016C00011E00E940F19E4E9FDE30E94F9188FEB85
:1016D00018E00E940F19A8EFB3E0E0E7F0E00E94E5
:1016E000981C0E94F1180C94850C023011F00C9497
:1016F000A30B8FEF8093AB038FE711E00E940F19CC
:10170000E6EAFDE30E94F9188FEB18E00E940F193A
:10171000A8EFB3E0EEE6F0E00E94981C0E94F118FA
:1017200002E010E0AEE6B0E04D9155270E94D118DE
:10173000A3EBB3E00D931C930091B30341E0041BB2
:101740000CBF0C94850C033011F00C94D10B8FEF6F
:101750008093AB038FE711E00E940F19E8EBFDE3E4
:101760000E94F9188FEB18E00E940F19A8EFB3E060
:10177000EFE6F0E00E94981C0E94F11802E010E0F1
:10178000AFE6B0E04D9155270E94D118A3EBB3E02E
:101790000D931C930091B30341E0041B0CBF0C9408
:1017A000850C043011F00C94F00B0E94DA178FE7CF
:1017B00011E00E940F19EAECFDE30E94F9188FEB8B
:1017C00015E00E940F190E94081AABECB3E00E94CA
:1017D000F3188091AA038F7D8093AA030C94850C43
:1017E000053011F00C94180C0E94DA178FE711E005
:1017F0000E940F19ECEDFDE30E94F91800917100B1
:10180000013011F00C940E0C8FEB11E00E940F19B7
:10181000EEEEFDE30E94F9180C94160C8FEB11E02C
:101820000E940F19E0E0FEE30E94F9180C94850C69
:10183000063011F00C94380C0E94DA178FE711E093
:101840000E940F19E2E1FEE30E94F9188FEB14E009
:101850000E940F19A8EFB3E0E4E7F0E00E94981CA3
:101860000E94F118E4E2FEE30E94F9180C94850C42
:10187000073011F00C94570C0E94DA178FE711E033
:101880000E940F19EEE2FEE30E94F91884E90E941B
:101890006F19E8E3FEE30E94F9188FEB11E00E9454
:1018A0000F19ECEEFCE30E94F9180C94850C08303B
:1018B00011F00C946F0C0E94DA178FE711E00E9470
:1018C0000F19E0E4FEE30E94F9188FEB11E00E948B
:1018D0000F19ECEEFCE30E94F9180C94850C09300A
:1018E00011F00C94850C0E94DA178FE711E00E942A
:1018F0000F19E6E7FCE30E94F9188FEB11E00E9454
:101900000F19ECEEFCE30E94F9180895ABEBB3E07D
:101910008C918F5F8C930091BB03013180E010F0BC
:1019200009F081E08F930091BB03013081E008F062
:1019300080E09F91892B882311F40C94A20C81E004
:101940008093BB030E94C40C0895ABEBB3E08C9171
:1019500081508C930091BB03013081E008F080E05E
:101960008F930091BB03013180E010F009F081E01A
:101970009F91892B882311F40C94C10C81E18093F1
:10198000BB030E94C40C08950E94DA170E9400193C
:101990008FE711E00E940F19ABEBB3E00D91112717
:1019A00041E150E00E94491BA6E8B0E0A00FB11F42
:1019B0000E94F3180091BB03053081E009F080E03C
:1019C0008F930091BB03083081E009F080E09F9184
:1019D000892B8F930091BB030B3081E009F080E0ED
:1019E0009F91892B8F930091BB030E3081E009F00A
:1019F00080E09F91892B8F930091BB03013181E09F
:101A000009F080E09F91892B882311F40C941E0D1E
:101A10008FEB18E00E940F19A8EFB3E0EBEBF3E0B7
:101A2000A190BB24E3E7F0E0AA0CBB1CEA0DFB1D70
:101A30000E94891C0E94F1180C94360D8FEB13E064
:101A40000E940F19A8EFB3E0EBEBF3E0A190BB24E9
:101A5000E3E7F0E0AA0CBB1CEA0DFB1D0E94891C09
:101A60000E94F118E2E5FEE30E94F9180895ABEB3D
:101A7000B3E08C918F5F8C930091BB03033080E0C7
:101A800010F009F081E08F930091BB03013081E0F9
:101A900008F080E09F91892B882311F40C94530D5A
:101AA00081E08093BB030E94750D0895ABEBB3E01A
:101AB0008C9181508C930091BB03013081E008F040
:101AC00080E08F930091BB03033080E010F009F0B9
:101AD00081E09F91892B882311F40C94720D83E08F
:101AE0008093BB030E94750D08950E94DA17009140
:101AF000BB03013011F00C94870D8FE711E00E94B9
:101B00000F19EEE2FDE30E94F9180C94A10D0230CA
:101B100011F00C94950D8FE711E00E940F19E0E78A
:101B2000FDE30E94F9180C94A10D033011F00C9400
:101B3000A10D8FE711E00E940F19ECE5FEE30E9472
:101B4000F9188FEB11E00E940F19E2E8FDE30E9403
:101B5000F9180895ABEBB3E08C918F5F8C930091F3
:101B6000BB03033680E010F009F081E08F93009111
:101B7000BB03013081E008F080E09F91892B88232E
:101B800011F40C94C60D81E08093BB030E94E80D14
:101B90000895ABEBB3E08C9181508C930091BB0323
:101BA000013081E008F080E08F930091BB030336A1
:101BB00080E010F009F081E09F91892B882311F4D7
:101BC0000C94E50D83E68093BB030E94E80D089515
:101BD0000E94DA170E9400198FE711E00E940F1986
:101BE000EEEFFCE30E94F91884E90E946F19EEE61B
:101BF000FEE30E94F918A8EFB3E0EBEBF3E00E94DC
:101C0000981C0E94F11840E050E060E070E0ABEBFF
:101C1000B3E0AD90BB24A4EBB1E0AA0CBB1CAA0CB2
:101C2000BB1CAA0DBB1D0D911D912D913C910E94D5
:101C3000761C0CF402C00C94270E8FEB11E00E946E
:101C40000F19E6E7FEE30E94F9180C948B0E40E8AA
:101C500051E561E070E0ABEBB3E0AD90BB24A4EBE9
:101C6000B1E0AA0CBB1CAA0CBB1CAA0DBB1D0D919C
:101C70001D912D913C910E94761C0CF402C00C9495
:101C8000590E8FEB15E00E940F19EBEBF3E0A190DA
:101C9000BB24E4EBF1E0AA0CBB1CAA0CBB1CEA0DB4
:101CA000FB1DA8EFB3E00E94411B0E94F1180C94A9
:101CB0008B0E8FEB13E00E940F19EBEBF3E0A1907A
:101CC000BB24E4EBF1E0AA0CBB1CAA0CBB1CEA0D84
:101CD000FB1DA8EFB3E00E94411B0E94F118E8E849
:101CE000FEE30E94F918EBEBF3E0A190BB24E4EBD8
:101CF000F1E0AA0CBB1CAA0CBB1CEA0DFB1D0E9448
:101D0000C71A002F112FA8EFB3E0E0E1F0E00E9426
:101D1000891C0E94F118089580E08093B00300911F
:101D2000B203013011F00C94310F0091BB0301306C
:101D300011F00C94AD0EA0E7B0E08C91A2E6B0E0FB
:101D40008D9388278D938D938C93AAE6B0E0EAE07B
:101D5000FAE30E949E1B0C942F0F0091BB030230EC
:101D600011F00C94C90EAEE6B0E08C91A2E6B0E0A2
:101D70008D9388278D938D938C93AFE6B0E08C91F3
:101D8000AAE6B0E08D9388278D938D938C930C9465
:101D90002F0F0091BB03033011F00C94E10EAFE65E
:101DA000B0E08C91A2E6B0E08D9388278D938D935F
:101DB0008C93AAE6B0E0EEE0FAE30E949E1B0C943E
:101DC0002F0F0091BB03043011F00C94010FECEBCA
:101DD000F3E00E94CB1AA2E6B0E00D931D932D9381
:101DE0003D9380E08093B1038091AA038062809349
:101DF000AA03AAE6B0E0E2E1FAE30E949E1B0C947B
:101E00002F0F0091BB03053011F00C94190FA1E7BF
:101E1000B0E08C91A2E6B0E08D9388278D938D93EE
:101E20008C93AAE6B0E0E6E1FAE30E949E1B0C94D4
:101E30002F0F0091BB03063011F00C942F0FA4E775
:101E4000B0E08C91A2E6B0E08D9388278D938D93BE
:101E50008C93AAE6B0E0EAE1FAE30E949E1B0C94A0
:101E60000510023011F00C945E0FABEBB3E0AD90B7
:101E7000BB24A3E7B0E0AA0CBB1CAA0DBB1D8D912F
:101E80009C91A2E6B0E08D939D9388278D938C93CF
:101E90000091BB03023011F00C94560FAAE6B0E09B
:101EA000EEE1FAE30E949E1B0C945C0FAAE6B0E000
:101EB000E2E2FAE30E949E1B0C940510033011F03D
:101EC0000C940510ABEBB3E0AD90BB24A4EBB1E0F8
:101ED000AA0CBB1CAA0CBB1CAA0DBB1D0D911D910D
:101EE0002D913C91A2E6B0E00D931D932D933C9370
:101EF0000091BB03013018F011F00C94810F0C9489
:101F0000BB0FABEBB3E0AD90BB24A0EBB1E0AA0CF0
:101F1000BB1CAA0CBB1CAA0DBB1D0D911D912D91C4
:101F20003C9149E050E060E070E00E946C1CA6E645
:101F3000B0E00D931D932D933D93A6E6B0E04D9137
:101F40005D916D917C91A2E6B0E00D911D912D9176
:101F50003C910E94761C0CF402C00C94BB0FA6E6C8
:101F6000B0E00D911D912D913C91A2E6B0E00D9352
:101F70001D932D933C930091BB03033681E009F040
:101F800080E08F934FEF5FEF6FEF7FEFABEBB3E04E
:101F9000AD90BB24A8EBB1E0AA0CBB1CAA0CBB1CE7
:101FA000AA0DBB1D0D911D912D913C910E94761C97
:101FB00081E009F080E09F91892B882311F40C9433
:101FC000E90FAAE6B0E0E6E2FAE30E949E1B0C9459
:101FD0000510ABEBB3E0AD90BB24A8EBB1E0AA0CCD
:101FE000BB1CAA0CBB1CAA0DBB1D0D911D912D91F4
:101FF0003C914AE050E060E070E00E94711CAAE66B
:10200000B0E00D931D932D933D93A0E3B0E00C91B0
:1020100002FB81E00EF080E08F93AAE6B0E04D91E4
:102020005D916D917C91A2E6B0E00D911D912D9195
:102030003C910E94761C80E00CF481E09F91892302
:10204000882311F40C9421110091B003053010F095
:102050000C943E10A2E6B0E00D911D912D913C91A3
:1020600041E050E060E070E00E946C1CA2E6B0E04D
:102070000D931D932D933D930C94D2100091B003BA
:102080000A3010F00C945810A2E6B0E00D911D91AA
:102090002D913C914AE050E060E070E00E946C1CA1
:1020A000A2E6B0E00D931D932D933D930C94D210B6
:1020B0000091B0030F3010F00C947210A2E6B0E063
:1020C0000D911D912D913C914CE350E060E070E04A
:1020D0000E946C1CA2E6B0E00D931D932D933D93DE
:1020E0000C94D2100091B003043110F00C948C10B9
:1020F000A2E6B0E00D911D912D913C9148E552E092
:1021000060E070E00E946C1CA2E6B0E00D931D93AD
:102110002D933D930C94D2100091B003093110F02F
:102120000C94A610A2E6B0E00D911D912D913C916A
:1021300040E15EE060E070E00E946C1CA2E6B0E06E
:102140000D931D932D933D930C94D2100091B003E9
:102150000E3110F00C94C010A2E6B0E00D911D916C
:102160002D913C9140EA5CE860E070E00E946C1CBC
:10217000A2E6B0E00D931D932D933D930C94D210E5
:10218000A2E6B0E00D911D912D913C9140E851E502
:1021900061E070E00E946C1CA2E6B0E00D931D931C
:1021A0002D933D93AAE6B0E04D915D916D917C91A8
:1021B000A2E6B0E00D911D912D913C910E94761CFC
:1021C0001CF011F00C94E6100C94F210AAE6B0E0AA
:1021D0000D911D912D913C91A2E6B0E00D931D93C0
:1021E0002D933C930091B203013081E009F080E02F
:1021F0008F930091BB03043081E009F080E09F9150
:1022000089238F93AAE6B0E04D915D916D917C9109
:10221000A2E6B0E00D911D912D913C910E94761C9B
:1022200081E009F080E09F918923882311F40C94C8
:102230001D11A2E6B0E00E94B01B0E94A8130C94EE
:1022400005108091AA038F7D8093AA03089580E0F2
:102250008093B0030091B203013011F00C94C611C9
:102260000091BB03013011F00C944611A0E7B0E0DF
:102270008C91A2E6B0E08D9388278D938D938C93FB
:10228000A6E6B0E00E94B01B0C94C4110091BB0301
:10229000023011F00C945C11AEE6B0E08C91A2E635
:1022A000B0E08D9388278D938D938C93A6E6B0E054
:1022B0000E94B01B0C94C4110091BB03033011F0B9
:1022C0000C947811AFE6B0E08C91A2E6B0E08D936B
:1022D00088278D938D938C93AEE6B0E08C91A6E623
:1022E000B0E08D9388278D938D938C930C94C411BB
:1022F0000091BB03043011F00C949811ECEBF3E067
:102300000E94CB1AA2E6B0E00D931D932D933D934E
:1023100080E08093B1038091AA0380628093AA0336
:10232000A6E6B0E0E6E0FAE30E949E1B0C94C4111E
:102330000091BB03053011F00C94AE11A1E7B0E0A1
:102340008C91A2E6B0E08D9388278D938D938C932A
:10235000A6E6B0E00E94B01B0C94C4110091BB0330
:10236000063011F00C94C411A4E7B0E08C91A2E601
:10237000B0E08D9388278D938D938C93A6E6B0E083
:10238000E6E1FAE30E949E1B0C946512023011F004
:102390000C94E311ABEBB3E0AD90BB24A3E7B0E04A
:1023A000AA0CBB1CAA0DBB1D8D919C91A2E6B0E0AE
:1023B0008D939D9388278D938C93A6E6B0E00E9421
:1023C000B01B0C946512033011F00C946512ABEB4A
:1023D000B3E0AD90BB24A4EBB1E0AA0CBB1CAA0CEB
:1023E000BB1CAA0DBB1D0D911D912D913C91A2E628
:1023F000B0E00D931D932D933C930091BB030130EE
:1024000081E009F080E08F934FEF5FEF6FEF7FEF98
:10241000ABEBB3E0AD90BB24A0EBB1E0AA0CBB1CCE
:10242000AA0CBB1CAA0DBB1D0D911D912D913C91B9
:102430000E94761C81E009F080E09F91892B88231F
:1024400011F40C942B12A6E6B0E0E6E0FAE30E9449
:102450009E1B0C946512ABEBB3E0AD90BB24A0EBDC
:10246000B1E0AA0CBB1CAA0CBB1CAA0DBB1D0D9194
:102470001D912D913C9149E050E060E070E00E9498
:102480006C1CA6E6B0E00D931D932D933D93A6E63C
:10249000B0E04D915D916D917C91A2E6B0E00D911F
:1024A0001D912D913C910E94761C0CF402C00C945D
:1024B0006512A6E6B0E00D911D912D913C91A2E62A
:1024C000B0E00D931D932D933C93A0E3B0E00C91ED
:1024D00001FB81E00EF080E08F93A6E6B0E04D9125
:1024E0005D916D917C91A2E6B0E00D911D912D91D1
:1024F0003C910E94761C80E014F009F081E09F91ED
:102500008923882311F40C94A2130091B0030530A1
:1025100010F00C949F12A2E6B0E00D911D912D9148
:102520003C9141E050E060E070E00E94711CA2E646
:10253000B0E00D931D932D933D930C9433130091B4
:10254000B0030A3010F00C94B912A2E6B0E00D917D
:102550001D912D913C914AE050E060E070E00E94B6
:10256000711CA2E6B0E00D931D932D933D930C9446
:1025700033130091B0030F3010F00C94D312A2E685
:10258000B0E00D911D912D913C914CE350E060E045
:1025900070E00E94711CA2E6B0E00D931D932D9394
:1025A0003D930C9433130091B003043110F00C945C
:1025B000ED12A2E6B0E00D911D912D913C9148E500
:1025C00052E060E070E00E94711CA2E6B0E00D9362
:1025D0001D932D933D930C9433130091B003093157
:1025E00010F00C940713A2E6B0E00D911D912D910F
:1025F0003C9140E15EE060E070E00E94711CA2E668
:10260000B0E00D931D932D933D930C9433130091E3
:10261000B0030E3110F00C942113A2E6B0E00D913E
:102620001D912D913C9140EA5CE860E070E00E94D1
:10263000711CA2E6B0E00D931D932D933D930C9475
:102640003313A2E6B0E00D911D912D913C9140E82D
:1026500051E561E070E00E94711CA2E6B0E00D93CC
:102660001D932D933D930091B203033011F00C9410
:102670005313A6E6B0E04D915D916D917C91A2E679
:10268000B0E00D911D912D913C910E94761C1CF0A3
:1026900011F00C945113A2E6B0E0E6E0FAE30E94D8
:1026A0009E1B0C947113A6E6B0E04D915D916D9167
:1026B0007C91A2E6B0E00D911D912D913C910E947C
:1026C000761C0CF402C00C947113A6E6B0E00D91D8
:1026D0001D912D913C91A2E6B0E00D931D932D9399
:1026E0003C930091B203013081E009F080E08F93C8
:1026F0000091BB03043081E009F080E09F918923C1
:102700008F93A6E6B0E04D915D916D917C91A2E62C
:10271000B0E00D911D912D913C910E94761C81E0BD
:1027200009F080E09F918923882311F40C949E1373
:10273000A2E6B0E0E2E1FAE30E949E1B0E94A81329
:102740000C9465128091AA038F7D8093AA0308954B
:102750008FEB11E00E940F19ECE8FEE30E94F918DC
:102760000091B203013011F00C9450140091BB039E
:10277000043011F00C94E713A2E6B0E00D911D9126
:102780002D913C91A1EBB3E04C915527662777271B
:102790000E946C1CA2E6B0E00D931D932D933D9317
:1027A00080E08093B103E2E6F0E0ABECB3E00E949E
:1027B000411B0E94111A8FEB15E00E940F190E9415
:1027C000081AABECB3E00E94F3180C944E140530D9
:1027D00011F00C940E1441E050E060E070E0A2E6CD
:1027E000B0E00D911D912D913C910E94761C11F04D
:1027F0000C9404148FEB11E00E940F19EEEEFDE330
:102800000E94F9180C940C148FEB11E00E940F1920
:10281000E0E0FEE30E94F9180C944E14063011F02B
:102820000C9424148FEB14E00E940F19A8EFB3E06E
:10283000E2E6F0E00E948C1C0E94F118E4E2FEE364
:102840000E94F9180C944E140091BB03073081E0EC
:1028500008F480E08F930091BB03083081E010F012
:1028600009F080E09F918923882311F40C9442148D
:102870008FEB11E00E940F19ECEEFCE30E94F918B7
:102880000C944E148FEB18E00E940F19A8EFB3E0E0
:10289000E2E6F0E00E948C1C0E94F1180C940015F6
:1028A0000091B203023011F00C94A4140091BB0308
:1028B000053081E009F080E08F930091BB03083080
:1028C00081E009F080E09F91892B8F930091BB03F9
:1028D0000B3081E009F080E09F91892B8F9300916C
:1028E000BB030E3081E009F080E09F91892B8F932C
:1028F0000091BB03013181E009F080E09F91892BB9
:10290000882311F40C9492148FEB18E00E940F1995
:10291000A8EFB3E0E2E6F0E00E948C1C0E94F11800
:102920000C94A2148FEB13E00E940F19A8EFB3E0F0
:10293000E2E6F0E00E948C1C0E94F118E2E5FEE362
:102940000E94F9180C9400150091B203033011F0A5
:102950000C94001540E050E060E070E0A2E6B0E0CA
:102960000D911D912D913C910E94761C0CF402C09A
:102970000C94C4148FEB11E00E940F19E6E7FEE3FC
:102980000E94F9180C94001540E851E561E070E0F0
:10299000A2E6B0E00D911D912D913C910E94761C14
:1029A0000CF402C00C94E2148FEB15E00E940F1996
:1029B000E2E6F0E0A8EFB3E00E94411B0E94F118AC
:1029C0000C9400158FEB13E00E940F19E2E6F0E083
:1029D000A8EFB3E00E94411B0E94F118E8E8FEE373
:1029E0000E94F918E2E6F0E00E94C71A002F112FAA
:1029F000A8EFB3E0E0E1F0E00E94891C0E94F1182A
:102A00000091B203013011F00C947C150091BB03CE
:102A1000013011F00C9416150E94DA1780916200B3
:102A2000809370000E9437180C947A150091BB03B4
:102A3000023011F00C9436158FEF8093AB03809128
:102A4000620080936E0002E010E0AEE6B0E04D91CF
:102A500055270E94D118A3EBB3E00D931C9300916E
:102A6000B30341E0041B0CBF0C947A150091BB0327
:102A7000033011F00C9456158FEF8093AB038091C7
:102A8000620080936F0002E010E0AFE6B0E04D918D
:102A900055270E94D118A3EBB3E00D931C9300912E
:102AA000B30341E0041B0CBF0C947A150091BB03E7
:102AB000043011F00C9460150E94DA170C947A150A
:102AC0000091BB03053011F00C946E150E94DA17CB
:102AD00080916200809371000C947A150091BB0381
:102AE000063011F00C947A150E94DA17809162007A
:102AF000809374000C94B015023011F00C9494156E
:102B00000E94DA17A2E6B0E08D919C91ABEBB3E0A6
:102B1000AD90BB24A3E7B0E0AA0CBB1CAA0DBB1D63
:102B20008D939C930C94B015033011F00C94B01558
:102B30000E94DA17A2E6B0E00D911D912D913C9113
:102B4000ABEBB3E0AD90BB24A4EBB1E0AA0CBB1C93
:102B5000AA0CBB1CAA0DBB1D0D931D932D933C937A
:102B600084E690E00E94F9190895ABEBB3E08C91F4
:102B70008F5F8C930E94BF150E94E6150895ABEB02
:102B8000B3E0AD90BB24A3E7B0E0AA0CBB1CAA0D38
:102B9000BB1D0D911C91003050E0150781E009F03C
:102BA00080E08F930091BB03013181E008F080E069
:102BB0009F918923882311F40C94E515ABEBB3E0C6
:102BC0008C918F5F8C930C94BF150895ABEBB3E0A1
:102BD000AD90BB24A3E7B0E0AA0CBB1CAA0DBB1DA3
:102BE0008D919C91A0E6B0E08D939C930E9400197A
:102BF0008FE711E00E940F19ABEBB3E00D911127A5
:102C000041E150E00E94491BA6E8B0E0A00FB11FCF
:102C10000E94F3188FEB11E00E940F19A8EFB3E0A8
:102C2000E0E6F0E00E94891C0E94F118ECE2FDE36E
:102C30000E94F9188FEB17E00E940F19A8EFB3E07C
:102C4000ECEAF3E00E94891C0E94F118EEE9FEE331
:102C50000E94F9188FEB1CE00E940F198AE10E9474
:102C60006F19A8EFB3E0EEEAF3E00E94891C0E941E
:102C7000F118089582E08093BB03A7E7B0E00D91BF
:102C80001C91003050E0150780E010F009F081E061
:102C90008F9300917100013081E009F080E09F91F5
:102CA0008923882311F40C9490160E94E6150E9443
:102CB000FF17A0E6B0E00D911C91003050E0150721
:102CC00080E010F009F081E08F93AAEAB3E08C91E4
:102CD00087FB81E00EF080E09F918923882311F427
:102CE0000C9490168B98AAEAB3E09C9192FF04C0D2
:102CF000839910C09B7F9C93839B0CC084E69F9319
:102D000099270E94F9199F91839B04C094609C931A
:102D10000E94311884E690E00E94F9190C9459162B
:102D20000895A0E6B0E00D911C91003050E0150729
:102D300080E010F009F081E08F93AAEAB3E08C9173
:102D400087FB81E00EF080E09F918923882311F4B6
:102D50000C94C8168B98AAEAB3E09C9192FF04C029
:102D6000839910C09B7F9C93839B0CC084E69F93A8
:102D700099270E94F9199F91839B04C094609C93AA
:102D80000E94311884E690E00E94F9190C94911683
:102D900084E690E00E94F919C798C49808950091BC
:102DA000AB030F3F11F00C94D81600000C940717DA
:102DB0000091AB03053010F00C94F616ABEAB3E0CB
:102DC0008C918F5F8C9302E010E0AFE6B0E04D9104
:102DD00055270E94D118A9EBB3E00D931C930091E5
:102DE000B90341E0041B0CBF0C94071702E010E08C
:102DF000AEE6B0E04D9155270E94D118A9EBB3E0A3
:102E00000D931C930091B90341E0041B0CBFAAEA87
:102E1000B3E08C9186FB16F00C943717A2E7B0E074
:102E20000D911C914CE350E00E94B718A9EBB3E060
:102E30004D935C93A4E7B0E04D915527A9EBB3E027
:102E40000D911C910417150710F40C942B170C947A
:102E50003C030C943717A2E7B0E00D911C9141E0C0
:102E600050E0040F151FA2E7B0E00D931C93A0EBF8
:102E7000B3E08C918F5F8C930091B203013081E0BD
:102E800009F080E08F930091BB03043081E009F0EA
:102E900080E09F918923882311F40C946517A1EB9E
:102EA000B3E08C918F5F8C93AAEAB3E08C9185FBA1
:102EB00016F40C9465178FEB15E00E940F190E9411
:102EC000081AABECB3E00E94F3180091B20304308F
:102ED00081E009F080E08F930091BB03003080E037
:102EE00010F009F081E09F918923882311F40C945C
:102EF000AB17A0E6B0E00D911C91003050E0150733
:102F000018F011F00C9486170C94AB17A0E6B0E003
:102F10000D911C9141E050E0041B150BA0E6B0E0C0
:102F20000D931C930091BB03013018F011F00C9429
:102F30009B170C94AB178FEB11E00E940F19A8EFB1
:102F4000B3E0E0E6F0E00E94891C0E94F118E0EA9C
:102F5000FEE30E94F9180091B203053011F00C94C1
:102F6000BD17A0E6B0E00D911C9141E050E0040FC8
:102F7000151FA0E6B0E00D931C930895A0E3B0E008
:102F80000C9103FB0EF406C084E690E00E94F91950
:102F90000C94BE170895A0E3B0E00C9103FB0EF073
:102FA00008C00E94DA1784E690E00E94F9190C9498
:102FB000CB170895A2E7B0E00E94AE1B8091AA0350
:102FC00080648093AA0380E08093AB0302E010E06A
:102FD000AFE6B0E04D9155270E94D118A3EBB3E0C6
:102FE0000D931C930091B30341E0041B0CBF0895A3
:102FF000C49A84E690E00E94F919C79A0895C49A89
:1030000084E690E00E94F91987E0E0E5F3ECA8E39C
:103010000E94C01BC49808958AEF90E00E94F9199D
:10302000A0E3B0E00C9103FB0EF018C00E94DA1789
:103030008FE711E00E940F19E4EAFEE30E94F918FD
:103040008FEB11E00E940F19E6EBFEE30E94F918E6
:1030500084E690E00E94F9190C9410180E9400195F
:1030600008958091AA038F778093AA030895A0E71B
:10307000B0E00D9111274FE050E0040F151FA3EBB6
:10308000B3E00D931C93A3EBB3E00D911C914FE0C3
:1030900050E004231523A3EBB3E00D931C93A3EBA3
:1030A000B3E00D911C9140E750E0040F151FA3EB16
:1030B000B3E00D931C93A0E7B0E00C9111272227F9
:1030C00033274FE050E060E070E00E946C1CA5EBFD
:1030D000B3E00D931D932D933D9394E0A5EBB3E0E6
:1030E0000E94851BA5EBB3E00D911D912D913C91A4
:1030F00044E550E060E070E00E946C1CA5EBB3E09A
:103100000D931D932D933D9389E2EFD08091B303EE
:10311000ECD08091B503E9D088E2E7D00895F89427
:10312000FFCF09D00E94491B00FC10D0089503D0A6
:103130001ED001F8F9CF0024E89457FF02C009D04F
:10314000689400F80BD010F80124089502D009D03B
:103150000895509540954F5F5F4F0895E89417FF8D
:103160000895009510950F5F1F4F68940895352FAF
:10317000242FE894452B11F468940895512F402F83
:103180000027112780E1440F551F001F111F021B4C
:10319000130B416018F4020F131F4E7F8A9599F7A5
:1031A000089514D081F0002E112E415050400ED0C1
:1031B00009F408954F935F93402D512D0E94491BB0
:1031C0005F914F91F2CF01E0112708958827842B5A
:1031D000852B08958F938D918823E9F711978F910F
:1031E0000895A8EFB3E08D91882311F078D0FBCF3C
:1031F00008950E94961B802D11F071D0FACF08958A
:1032000081E073D015D080E870C08FE7213039F0AD
:103210008FEB223021F08FE8233009F08FEC810F03
:103220000C94751988EE93E0E4D03197D9F708959E
:1032300083E09927DEC08AEF90E00E94F919D79ABF
:10324000D69AD59AD49AD39AD29ADA9885E090E011
:103250000E94F919DB98DF98DE98DD9ADC9ADB9AF8
:10326000EF93FF93E5E1F0E00E94ED19FF91EF91FC
:10327000DB98BCD0DB9AEF93FF93E5E1F0E00E948E
:10328000ED19FF91EF91DB98B1D0DB9AEF93FF93AB
:10329000E5E1F0E00E94ED19FF91EF91DB98A6D0F7
:1032A000DC98DB9AEF93FF93E5E1F0E00E94ED19E3
:1032B000FF91EF91DB989AD089E217D084E115D085
:1032C00085E513D08DE611D088E70FD088E20DD0C8
:1032D00088E20BD08EE009D086E007D00895DA9A14
:1032E000829505D004D082D00895DA98F9CF8595DB
:1032F00010F4DC9A01C0DC98859510F4DD9A01C0C9
:10330000DD98859510F4DE9A01C0DE98859510F45D
:10331000DF9A01C0DF98DB9AEF93FF93E5E1F0E0DD
:103320000E94ED19FF91EF91DB98089500FC05D004
:10333000089530D005D001F8F9CF37D03FD00895A7
:10334000842F952FA62FB72FE894452B462B472B7C
:1033500011F468940895402F512F622F732F002786
:10336000112722273327F0E2440F551F661F771FCE
:10337000001F111F221F331F081B190B2A0B3B0BA9
:10338000416028F4080F191F2A1F3B1F4E7FFA9532
:1033900059F708950024E89477FF02C006D0689496
:1033A00000F809D010F80124089512D04F5F5F4F44
:1033B0006F4F7F4F0895E89437FF0895009510955B
:1033C000209530950F5F1F4F2F4F3F4F6894089502
:1033D000409550956095709508953197F1F708954F
:1033E000689462F80895E89462F8089581E090E0A6
:1033F00000C0EF93FF93EE27E82BE92B31F0EAEFC3
:10340000F0E03197F1F70197D1F7FF91EF9108952F
:10341000A2ECB3E0EFEBF3E00E943D1A33970C947B
:103420002B1AEBECF3E0ACEBB3E00E94191AADE021
:10343000BB27868197810E94D61B0D93838194813F
:103440000E94D61B0D93808191810E94D61B0D9303
:103450000895EDE0FF2782810E94CB1B8AE38D93C4
:1034600081810E94CB1B8AE38D9380810E94CB1BBC
:1034700088278C930895EDE0FF2781810E94CB1B64
:103480008CE58D9380810E94CB1B8CE58D9382818E
:103490000E94CB1B88278D93089593E0ADE002C076
:1034A00096E0AAE0B0E08FB7F89401910D939A9559
:1034B000E1F78FBF08950191119145EB55E00E940E
:1034C0009718440F440FF42E0F31150728F481E0AC
:1034D000E82E0395D02E22C00C33150728F482E085
:1034E000E82E0E51D02E1AC00150150B4DE651E0BA
:1034F0000E94B718F40E7CE07A95872F9927EEE1A9
:10350000F5E3A2E1BB270E94A61B02171307A0F355
:103510007395E72E021B130B0395D02E0895000020
:103520001F003B005A0078009700B500D400F3005C
:10353000110130014E01019111912191308140E83A
:1035400051E561E070E00E949919042F152F0C9449
:103550005D1AA3DF0E2D0A95802F0295003220F010
:103560001F2D137009F40395DA940D0D1127992777
:10357000E2E8F5E3A8E1BB270E94AB1B080F111F8F
:103580000895000F1B2A384755647381909E0E944E
:103590009B1A0C94AA1A81DF0F2D11274CE3552793
:1035A0000E94911855270E0D151F4CE32227332733
:1035B000662777270E94531B0D0D131F231F0895A5
:1035C0006CDFDF92EF92FF920F2D11272227332716
:1035D0004DE651E060E070E00E94531BFF904F2DDC
:1035E0004D5F469546955527662777270E946C1CA8
:1035F000EF90DF900F931F932F933F930E94AA1A8F
:10360000222733277F916F915F914F910C946C1C0F
:1036100047DFAF92BF92CF920E94E11A40E851E596
:1036200061E070E00E94531BFF90EF90DF900F93DA
:103630001F932F933F930E94CC1A7F916F915F91BC
:103640004F910C946C1C019111912191308140E8B3
:1036500051E561E070E00E9499190C94331B0191CF
:1036600011912191308140E15EE060E070E00E94C4
:103670009919F42E4CE350E00E949718E42ED02EB6
:103680000895AF93BF930E94231BBF91AF910C94F9
:10369000291A0F92B801469F8001479F100D569F2F
:1036A000100D0F9008950F921F922F92C801D9010B
:1036B000489F80014A9F90014B9F202C499F100DED
:1036C000211D321D5A9F202C589F100D211D321D87
:1036D000599F200D311D689F200D311D699F300DB0
:1036E000789F300D2F901F900F9008950E94961B89
:1036F0000D920020D9F70895369A3699FECF369A62
:103700003699FECF84B195B10895903071F00D9146
:103710001D912D913C9136952795179507959A9572
:10372000D1F73C932E931E930E930895C89531962E
:103730000020089591E005C092E003C094E001C02C
:1037400098E0F4DF0D929A95E1F70895880F991F9C
:10375000E80FF91FF1CFE80FF91FECCF82E001C0AD
:1037600084E099279D938A95E9F7089591E088234D
:1037700021F08894991F8A95E9F7892F90950895EB
:10378000BB270E94B61B9C9198279C933197F1F719
:1037900098279C93089500278A3018F08A50039543
:1037A000FBCF005D0D93805D8D9308958053905302
:1037B0000027813018F0065F8A95FBCF090F089526
:1037C000AF93BF930F939F938F938FB78F93ACEB70
:1037D000B3E08C9183958D938C3309F03DC088279D
:1037E0008E9311968C9183958D938C3309F034C010
:1037F00088278E9311968C9183958D93883161F5EE
:1038000088278E9311968C9183958D939C910EE1D0
:10381000943089F0963079F0993069F09B3059F006
:103820000CE1923039F411969C911197937019F430
:10383000039501C00FE1801778F071F081E08E935D
:1038400011968C9183958D938D3031F481E08E9318
:1038500011968C9183958C938F918FBF8F919F91AF
:103860000F91BF91AF910F921F922F923F924F9263
:103870005F927F92AF92BF920F931F932F933F93CC
:103880004F935F936F937F938F939F93AF93BF9368
:10389000CF93DF93EF93FF938FB78F930E94CF1651
:1038A0008F918FBFFF91EF91DF91CF91BF91AF913A
:1038B0009F918F917F916F915F914F913F912F9148
:1038C0001F910F91BF90AF907F905F904F903F906E
:1038D0002F901F900F901895040F151F261F371F4C
:1038E0000895041B150B260B370B089504171507B5
:1038F000260737070895000F111F221F331F089551
:1039000000951095209530950F5F1F4F2F4F3F4F1B
:103910000895019110810EC0019111912191308182
:103920000BC00191108117FF05C03FEF2FEF04C0BE
:10393000008111272227332737FF03C0E1DF8DE203
:103940008D93CF93DF93CF92DF92EF92AA24BB2483
:10395000CC24DD24EE2440E2CAE0DD2755E093E3E9
:103960008881890F87FD9F7083FD907F891B8993D4
:103970005A95A9F7C0DFAA1CBB1CCC1CDD1CEE1C91
:103980004A9551F7E894EFE0FF2782910ED0EB3093
:10399000E0F71EF068948A2D0CD088278D93EF9065
:1039A000DF90CF90DF91CF910895982F829501D02D
:1039B000892F8F70805D26F0803309F40895689414
:1039C0008D930895E199FECFEEBBFFBB319608952C
:1039D00091E001C092E07B3751F47FB7F894F2DFB9
:1039E0008D918DBBE29AE19A9A95C9F77FBF7727AF
:1039F000089591E001C092E0E5DFE09A8DB38D93E8
:103A00009A95D1F70895FFFFFFFF0F00000008000F
:103A100000007F51010001000000630000001D0054
:103A200000000F270000FF84E201556E6976657281
:103A300073616C2054696D657220000062792050BA
:103A4000697420262054542032303037000020453D
:103A5000696E7374656C6C756E67656E202000000E
:103A60002050726F6772616D6D7A656974656E2042
:103A700000002020205A65697470756E6B74652093
:103A8000202000006175746F6D2E204175736C00ED
:103A900073656E200000206D616E2E204175736C81
:103AA000000073656E2020007A656974672E2041DE
:103AB00075736C005761727465206269732053746A
:103AC0006172742000005370696567656C766F726F
:103AD0006175736C2E20000050726F673120426553
:103AE0006C69636874756E67000050726F6731208F
:103AF00050617573652020202020000050726F6790
:103B0000312042696C6465722020202000005072D0
:103B10006F67322042656C69636874756E67000078
:103B200050726F673220506175736520202020200D
:103B3000000050726F67322042696C646572202009
:103B40002020000050726F67332042656C69636803
:103B500074756E67000050726F6733205061757323
:103B6000652020202020000050726F6733204269BA
:103B70006C64657220202020000050726F67342032
:103B800042656C69636874756E67000050726F6798
:103B90003420506175736520202020200000507271
:103BA0006F67342042696C64657220202020000019
:103BB00050726F67352042656C69636874756E6713
:103BC000000050726F6735205061757365202020AA
:103BD0002020000050726F67352042696C64657266
:103BE00020202020000020426174746572696520E5
:103BF0006C6565722021000020426974746520772D
:103C000065636873656C6E20000042617474657250
:103C100069652073636877616368000020204261F2
:103C2000747465726965204F4B20202000002020AD
:103C30007374617274652054696D65722020000090
:103C4000202054696D657220626572656974202058
:103C500000004D656E756520617573770000686CB6
:103C6000656E200054696D6572202043616E6F6E31
:103C700020454F530000205374616E646279204DDB
:103C80006F647573202000002053656B756E64654A
:103C90006E20000050726F6772616D6D2062656505
:103CA0006E64657400002057617274652000204ABC
:103CB00065747A742000576572746520676573694E
:103CC00063686572742000005A656974702E2067FD
:103CD000656C00007363687420002020466F6B756C
:103CE0007373696572656E202020000020202020FB
:103CF00020456E7465722020202020200000204185
:103D000075736C0073656E205374617274200000CB
:103D10002042656C6963687465002053746F70207D
:103D20006D697420456E7465722000007300206D0B
:103D3000697420466573747374656C6C2020000090
:103D4000456E74657220756E642068616C74656E72
:103D50000000204175666E61686D65206C007566B7
:103D6000742000002042656C69636874652000005F
:103D7000206F686E6520466573747374656C6C2083
:103D800000004D656E7565206F64657220456E7428
:103D90006572000020204C4344204B6F6E747261AA
:103DA000737420200000204C43442048656C6C69EB
:103DB000676B6569742000006D61782E2048656C22
:103DC0006C69676B6569742000002020556872205B
:103DD0007374656C6C656E202020000020205356A3
:103DE0004120616B746976203F2020200000202054
:103DF00020202020206A6120202020202020000078
:103E00002020202020206E65696E20202020202088
:103E1000000020506F7765722054696D656F75746E
:103E200020200000204D696E7574656E00005A6593
:103E30006974702E206C0000736368656E203F000B
:103E400057657274652073706569636865726E206A
:103E500000002053656B756E64656E0020696E739B
:103E60002048617570746D656E756520000073651E
:103E70007A65697420002020202020204E2F4120C8
:103E80002020202020200000202B000020202020A7
:103E900020202020202020202020202000006E0034
:103EA000732000002020426974746520546173748B
:103EB00065202020000020206C6F736C6173736597
:083EC0006E20212020200000EB
:00000001FF
